:020000040800F2
:10000000F01D0020A901000821150008410C00087E
:1000100000000000000000000000000000000000E0
:10002000000000000000000000000000991C000813
:10003000000000000000000023150008991D0008C2
:10004000BB010008BB010008BB010008BB010008A0
:10005000BB010008BB010008BB010008BB01000890
:1000600000000000BB010008BB010008BB01000844
:10007000BB010008BB010008BB0100080000000034
:10008000BB010008BB010008000000009D1E000825
:10009000D11E0008591F00087D1F0008BB01000881
:1000A000BB010008BB010008BB010008D11F00080C
:1000B00061200008000000000000000000000000B7
:1000C000BB01000800000000BB01000800F002F8BE
:1000D00000F03EF80CA030C8083824182D18671E10
:1000E000A246AB4654465D46AC4201D100F030F822
:1000F0007E460F3EB6460FCC0126334200D0FB1A97
:100100003343A246AB461847E04C0000004D0000C8
:10011000103A02D378C878C1FAD8520701D330C850
:1001200030C101D504680C60704700000023002432
:1001300000250026103A01D378C1FBD8520700D31E
:1001400030C100D50B6070471FB51FBD10B510BD85
:1001500000F090FB1146FFF7F7FF02F09FFD00F063
:10016000A8FB03B4FFF7F2FF03BC00F007FC00009C
:1001700070B505460C46164602E00FCC0FC5103E82
:10018000102EFAD2082E02D303CC03C5083E042E4B
:1001900007D301CC01C5361F03E021782970641C08
:1001A0006D1C761EF9D270BD07488047074800478E
:1001B000FEE7FEE7FEE7FEE7FEE7FEE70448054947
:1001C000054A064B70470000AD1D0008CD00000831
:1001D000F0150020F01D0020F0190020F01900207B
:1001E000F8B5042A2CD3830712D00B78491C03706E
:1001F000401C521E83070BD00B78491C0370401C17
:10020000521E830704D00B78491C0370401C521EF9
:100210008B079B0F05D0C91ADF002023DE1B08C9FE
:100220000AE0FFF7A5FFF8BD1D4608C9FD401C46C2
:10023000B4402C4310C0121F042AF5D2F308C91A87
:10024000521EF0D40B78491C0370401C521EEAD495
:100250000B78491C0370401C012AE4D40978017012
:10026000F8BD7047704770470246C80FC00781430A
:100270004B0030B54B405B009B0D20D01923DB06B3
:10028000C91801231B05994220DB0324A407042578
:100290001346AB400BD3002B04D1EB0613409B005D
:1002A000E34204D401246407002312195941FF23B7
:1002B0001B0599420BD2C9000143500F09E0CB0244
:1002C00004D501430803024305D0054830BDFF2192
:1002D000C905084330BD084607210905884330BDDC
:1002E0000000C07FF0B58B4C0F09254689B0BD4397
:1002F0007BD01D092646AE43FAD00E465E4027400D
:10030000F60F3E43254071D024012142FBD0FF244B
:10031000AD19A4042D1B039501252D05DB02DB0A75
:10032000C9022B43C90A29431E010901040F130FF7
:10033000050121431701880B820391432D098C4647
:10034000A90B1E438A039543B30B9A0396433F09B7
:10035000BA0B9403A74302962E467E430497B646F3
:100360004E19D7190C460196544305977E43371B07
:100370007646BF1B3601B646BE0B3619009676464A
:10038000BC043719009C01D3641C00946400002F46
:1003900001D001263443029E049F754366467E4386
:1003A0000496760034196E0034190094029C019E64
:1003B0001C196643751BAE46069465464519059C97
:1003C00005956C43594375460891691A0191049E3D
:1003D00001465143A41B0491611A009C0791E10658
:1003E00005D061090122114302E072E06EE061096B
:1003F000089D00272C0A2D066918049D7C412A0AB5
:100400002D066918019D6241AC0DAD026D18544175
:10041000079A910D920255196141029A6446584318
:100420005443069B059A5A43121A131B9A0E9B01BA
:100430005B187A41010B0005C3185141220A2006BE
:1004400044195A419A4200D2491C0120400281427B
:1004500003D315230226F64302E014230326F643B2
:100460002020C51AA9401746AF40DA400A4320466B
:100470000399D8400914731819055118039A384381
:10048000D2075140AC4009D00122944006D300224B
:10049000401C5141002C01D1400840001E4A9342AB
:1004A00012D3012203989206904207DB05204007F1
:1004B00009181A480143C012414004E003204007D4
:1004C0000818C10FC907002009B0F0BD0020F107CE
:1004D000FAE705180C464C4111486D42A04115D36E
:1004E00094181A465A410E48644290410ED3012096
:1004F0004A004005824209D35A00824206D359403D
:10050000C90F084AC90700201143DDE7002006494A
:10051000DAE700000000FF07FE070000FFFFFF7F93
:100520000000E0FF0000F07F0000F87F0121C90516
:100530000123411842001B06D3185B0E0AD0C110DC
:100540000722D206891840075242D14201D55200F3
:1005500089187047090208D50146002A03D0C10F47
:10056000C9070020704710467047420202D00020A1
:1005700002497047072109050143F4E70000F87FAD
:10058000F0B5FF252D04C609C209FF2704462E40F9
:100590000137CB093E4348402A402B400746002AFA
:1005A0006BD0002B69D0AA4267D0AB4265D000283F
:1005B00000DA32460125ED0529432C4309022002C9
:1005C000090AD21A4B0C7F24E31A434C000A7C44DC
:1005D000E35C7D242404121914145B00A2188842E1
:1005E00001D3521C00E0400049420C465C432411F8
:1005F0005C43DB016415E318040A5C43C502200D6B
:100600000C4644436419250A5D432303EC0C0D4654
:10061000654300030019EB184C42A34201D35B1859
:10062000401CD4052018002B07D05B00C91804D348
:10063000401C002901D1400840003F2189048A4222
:1006400009D3002A08DC1106090F04D00321490749
:100650004018C00FC007F0BD0122410012068918E2
:100660007F2252069142F6D205214907C84201D5A0
:100670009010F0BDFF20C005F0BD002F00DA32461B
:100680001648AA4207D2AB4205D21902090E17D06A
:10069000F80FC007F0BDFF2563002D06AB42F9D867
:1006A0004900A942F6D8AB4201D1A942F2D0A942F1
:1006B00001D1002101E061004908D0050843F0BDE7
:1006C0001102090EFBD0FF200243D005F0BD0A46FF
:1006D0000146104654E70000EE4400000000C07FD1
:1006E0000102C21504D00123DB071943002A0ADBEB
:1006F0009E239A1A02D40846D0407047FF22410038
:100700001206914201D900207047C017C0437047BC
:100710001F22030C02D10F2200041CD0030E01D1B2
:100720000002083A030F01D10001121F830F01D10B
:100730008000921E002801DB4000521ED205511895
:10074000021251181922904004D3491C002801D1EB
:100750004908490008467047C10FC90700D0404208
:10076000012292071143D3E701218907D0E7000056
:10077000F8B5264C4E00069DA6420AD8A64201D1E5
:10078000002806D15E00A64203D8A6420AD1002A5C
:1007900008D00D242404254233D02946002000F03F
:1007A00090F8F8BD0C461C4311D4994207D0C81AE2
:1007B00002D3EFF30080F8BDEFF30080F8BD801A9C
:1007C00002D3EFF30080F8BDEFF30080F8BD0924F9
:1007D0002407E5008B4207D0581A02D3EFF30080BC
:1007E00006E0EFF3008007E0101A03D3EFF3008078
:1007F000A04303E0EFF30080A043284380F3008888
:10080000F8BD009500F074F8F8BD00000000E0FFAE
:1008100010B5FF231B0644009C421DD84C009C428F
:100820001AD80346124A0B4307D4401A02D3EFF3F7
:10083000008010BDEFF3008010BD081A03D3EFF362
:100840000080904305E0EFF3008001219043C90749
:10085000084380F3008810BD0D231B041A4204D006
:100860001146002000F02DF810BD00F04BF810BD2F
:1008700000000090754600F04DF8AE460500694650
:100880005346C008C000854618B020B5FFF796FC57
:1008900060BCB64600260027C0C5C0C5C0C5C0C5DF
:1008A000C0C5C0C5C0C5C0C5403D490849008D464A
:1008B000704710B50446C046C0462046FFF751FCBD
:1008C00010BDC80212D54803400F002804D0C80349
:1008D000C043012188407047EFF300800001000908
:1008E00003210907084380F3008870470020704700
:1008F00010B500200249029A00F010F810BD000067
:100900000000F87F10B5024800F008F810BD0000A4
:100910000000C07F00487047A000002010B50C46C2
:100920001107090F092904D00A290AD008290CD176
:1009300004E011460820FFF7C4FF06E0510606D583
:1009400001E0510601D50120C007214610BDD106A6
:1009500007D501010909CC084907000E0006044328
:1009600009E0410F20024907000A0143200E00065A
:100970001D22D14101430846E7E700000149182044
:10098000ABBEFEE726000200704770B514460D4668
:100990000646200407D0B0B200F006F82870641EA6
:1009A0006D1C761CF5E770BD70B5044600F0D8F8F4
:1009B000A020214DA847214EB047200AA847B047A4
:1009C000E0B2A847B04700F0CBF8A120A847B04755
:1009D000002000F037F9044600F0E2F8204670BD30
:1009E00070B514460D460646200407D02978B0B2EB
:1009F00000F006F8641E6D1C761CF5E770BD000063
:100A0000F8B50C46054600F0ABF8A0200A4EB047FA
:100A10000A4FB847280AB047B847E8B2B047B847C6
:100A20002046B047B84700F0BBF80A20F8BC02BC2B
:100A30008E4600F083B8C046A90C00080D0D0008D2
:100A400080B500F013F800F0CFFF01F0E1F801F0FD
:100A500037F801F0A7F800F075FF01F003F800F097
:100A60002BFF80BC01BC864601F060B8F8B50020C1
:100A7000022101F071FB0A2000F060F8664D287930
:100A8000411973268C5D00F0B1F8844208D17420BE
:100A9000285C00022946743149784018286301E037
:100AA0000120687101240221204601F055FB0A2033
:100AB00000F044F8287941198F5D00F097F88742DB
:100AC00008D17420285C0002294674314978401806
:100AD000686300E06C711320022101F03DFB0A20E5
:100AE00000F02CF8287941198E5D00F07FF88642DD
:100AF00008D17420285C00022946743149784018D6
:100B0000A863F8BD6C71F8BD80B5C54841F200011D
:100B100002F07FF8411E884180BDC04674223E48E5
:100B200000217E2A02D08154521CFAE78170018094
:100B30007047C0462C4800214170704781B000903A
:100B400003480099016001680029FCD101B0704799
:100B50000C0D002081B00090009801B0704700009B
:100B6000F8B501F0E5F8E44C01262046314602F0E4
:100B70004CF802252046294602F047F8042738465B
:100B8000FFF7E8FF2046314602F03DF83846FFF710
:100B9000E1FF20462946F8BC04BC964602F033B873
:100BA000F8B501F0C5F8D44C02252046294602F0DC
:100BB0002AF801262046314602F025F80427384657
:100BC000FFF7C8FF2046294602F01FF820463146AD
:100BD00002F01BF83846F8BC02BC8E46FFF7BABFDD
:100BE000014840787047C04600010020B0B5401E63
:100BF0000021094B74240A46CDB2A84204DD5D19D8
:100C00002D5D5219491CF7E70C4801788918407886
:100C10000918FF208843B0BD3401002010B5401EE4
:100C20000021064B0A46CCB2A04203DD1C5D12191E
:100C3000491CF8E7FF20904310BDC046100D00206E
:100C4000FEE70000FEB5009001F06CF800210226DE
:100C5000012001900C46019D07291CD8A64F38465B
:100C60000291314601F0CFFF3046FFF773FF38465F
:100C7000314601F0CAFF3846294601F0CAFF27462F
:100C800004462846FFF766FF0299601E84417800FB
:100C90000419491CE0E7009810B101F005F801E0E3
:100CA00001F022F8E0B2FEBDFEB5044601F040F8C6
:100CB00091480226314601F0A6FF0027012001904D
:100CC000072F1FD860B2002802948B4D284603D40A
:100CD000019901F098FF02E0019901F096FF30467A
:100CE000094CA0472846314601F08FFF3046A04707
:100CF0002846314601F087FF3046A0477F1C029C02
:100D00006400DDE7FEBDC046550B000870B501F07C
:100D100009F8794C0221204601F077FF0125284689
:100D2000FFF718FF00262046294601F072FF30B178
:100D3000701CFA2E0646F6D3FFF732FF04E00221BC
:100D4000204601F060FF0025284670BD00F06AB81B
:100D5000FEB5A94802F0A0FF0920C60601210191B5
:100D60000025202730462A463B46A44CA0470322B4
:100D70000292A34C304629463B46A04730463946AE
:100D8000A04A90471027304601992A463B469B4C83
:100D9000A04730462946029A3B46994CA047304628
:100DA0003946984A90474027304601992A463B46A3
:100DB000924CA04730462946029A3B46904CA047A9
:100DC000304639468F4A90478027304601992A4657
:100DD0003B468A4CA04730462946029A3B46884CFF
:100DE000A04730463946874A90478348401C02F066
:100DF00053FF854E3046019C21462A4623467F4FAD
:100E0000B84730462946029A23467D4DA8473046CA
:100E100021467C4A03B0F0BC08BC9E461047C04641
:100E200000040048F8B51C4802F036FF1B4F0125AE
:100E30000024724E38462946224642F20003B0474B
:100E40006F4E38462146224642F20003B0473846EC
:100E500042F2000101F0D7FE0F48C01C02F01CFF57
:100E6000254E3046294622462B46644FB847304629
:100E7000214622462B46624FB84702273046294674
:100E800022463B465D4DA8473046214622463B461A
:100E90005B4CA047F8BDC0461305000000080048A1
:100EA000F8B5E14CA34D2046A847601CA847601D3B
:100EB000A847114E002401258023504F304621467B
:100EC0002A46B8474023304621462A46B8470920DB
:100ED000C606304621462A4641F20003B84730464E
:100EE00021462A4640F20013B847F24821462A46D6
:100EF00048F20003B847F8BD00140048B0B50D48EB
:100F000002F0CAFEEB4C0121002520462A4640F69D
:100F1000000301F083FE03222046294640F6000329
:100F200001F09BFE204640F60001B0BC04BC964692
:100F300001F069BE1205000070470000F0B585B0F1
:100F4000D94C204602F0A8FE601C02F0A5FE092044
:100F5000C40601260227D64D204631463A4648F2BD
:100F60000003A8470021039103220492244D204648
:100F700048F20003A847204648F20001214A904762
:100F8000CC4808250296314601973A462B46C84C74
:100F9000A047C8480399049A2B46194CA047C54C52
:100FA00020462946174A90471025204631463A46A2
:100FB0002B46BF4EB04720462746039E3146049A33
:100FC0002B460F4CA047384629460E4A904720250D
:100FD00038460299019A2B46B54CA047384631460F
:100FE000049A2B46064CA04738462946054A05B0C8
:100FF000F0BC08BC9E461047110500001D2C0008DF
:101000005B2C0008072C0008000400480C4800680E
:1010100040F2E831B0FBF1F0401E010E00D0FEE7D7
:101020000849094A5060094803680B4003218907B1
:101030005918016000209060072010607047C0467A
:1010400018000020FFFFFF0010E000E020ED00E0AE
:10105000F0B587B03648002141600E4601919349B2
:1010600040F210608847344D34492846884703AC25
:101070003349204688474720029020803148059018
:101080000496314A28462146904701272F4A284690
:10109000394600979047142002212D4A90472D4948
:1010A0002846884740F21060401C804988472A4EF5
:1010B00030462249884703AD28462149884702988F
:1010C000288020480590019C0494304629461E4AF9
:1010D0009047304639461D4A90471520032529463A
:1010E0001B4A904730461B49884740F21060801CDD
:1010F0006E498847194E30461049884703AF384635
:101100000F498847164838801648059004943046A1
:1011100039460D4A9047304600990C4A90471620B0
:1011200029460B4A904730460A49884707B0F0BD28
:1011300000010020993C000800400140353E0008B5
:10114000813F0008E7030000A93E00085D3F00085A
:101150009D3A00089F3E00080044014000480140BD
:101160001F1C00000F270000FEB502901C20022566
:10117000294602F093FC4C4802F08EFD0920C70678
:1011800001240426019638462146324601F010FD1E
:10119000384629462246334601F040FD00210091A1
:1011A00038462246334601F058FD08263846214687
:1011B000324601F0FDFC384629462246334601F00E
:1011C0002DFD3846009F39462246334601F045FD45
:1011D000164802F061FD164D284602F027FF28460A
:1011E000029902F0F1FE2846394602F099FF28469E
:1011F00041F2000102F0A9FF284640F2004102F04E
:101200007AFF2846019902F083FF2846314602F012
:1012100094FF284602F024FF0521284603B0F0BCC5
:1012200004BC964602F03ABF110500001107000009
:1012300000440040F8B51C4C1C4D2046A847641CD7
:101240002046A8472046A8470920C5060126184C75
:101250002846314632463346A04700240327284615
:1012600021463A46334601F0F8FCA04802253146B3
:101270002A4644F200030E4EB0479C4E30462146AB
:101280003A4644F2000301F0E8FC304621462A4683
:1012900041F20003064CA047304644F20001F8BC7E
:1012A00004BC964601F0B1BC11050000993C000851
:1012B0001D2C000800040048F8B500F035FF0A2492
:1012C0000F4E2046B04700F0FDFE2046B0470020FC
:1012D00002250C4A0C4F2946B8472046B04701204A
:1012E00029460246B8471320084A2946B8472046EF
:1012F000B04700F0FFFEF8BC01BC864600F008B81D
:101300003D0B0008040A00007D2100086504000070
:10131000FEB57020022100F01FFF3220FFF70EFC07
:101320006D4E3079811973240D5DFFF75FFC8542A6
:1013300007D17420305C000231467431497840187E
:10134000B0607120022100F007FF3220FFF7F6FBAA
:10135000307981190D5DFFF749FC854207D1742072
:10136000305C00023146743149784018F0607220D8
:10137000022100F0F1FE3220FFF7E0FB3079811905
:101380000D5DFFF733FC854207D17420305C00020D
:10139000314674314978401830610221204600F00E
:1013A000DBFE3220FFF7CAFB307981190D5DFFF7B4
:1013B0001DFC854207D17420305C00023146743137
:1013C00049784018706174250221284600F0C4FE57
:1013D0003220FFF7B3FB307981190F5DFFF706FC70
:1013E000874206D1705D0002314674314978401859
:1013F000B0617520022100F0AFFE3220FFF79EFBA6
:10140000307981190F5DFFF7F1FB874206D1705DDE
:1014100000023146743149784018F061762002218B
:1014200000F09AFE3220FFF789FB307981190F5DB9
:10143000FFF7DCFB874206D1705D00023146743154
:101440004978401830627720022100F085FE322072
:10145000FFF774FB307981190F5DFFF7C7FB8742F7
:1014600006D1705D000231467431497840187062CF
:101470006F20022100F070FE3220FFF75FFB307911
:1014800081190C5DFFF7B2FB844208D1705D000248
:1014900031467431497840180290B06201E0B06A78
:1014A0000290B068019037460C37BCCF306A00908C
:1014B000716A01988218D21812195219D21900981B
:1014C00010184018401E80B204494140F162029851
:1014D000091A48424841FEBD34010020FFFF0000C8
:1014E000F44840F6000101F092BBC04600040048F9
:1014F000032811D8094A1018C9B24A07D20F4271FD
:101500008A07D20F42700A07D20F4272CA06D20F60
:1015100042738906C90F41747047C046000000201D
:1015200070477047F0B58BB00020C04C0490214646
:1015300040F29012FFF729FA0894207808B10428A5
:1015400002D3BA4903200870B949087040F2F81074
:10155000B84908580A9040F2F4100858099040F22F
:10156000F0100A5840F2EC10085840F2E8140C59F8
:101570000B25EE43019608361827DEB1AB498D19CD
:10158000697DB940234604460A9808180A90204607
:101590001C46697CB940099BCB180993697BB9400B
:1015A0008A18697AB94008186979B9400C19083F56
:1015B000761CE2E740F2F8119E4E0A9F775040F207
:1015C000F411099D755040F2F011725040F2EC1187
:1015D000705040F2E813F450974E642C01D3B4429B
:1015E00001D99449CE50642802D39349884204D942
:1015F00040F2EC1064218F4C21509048824204D973
:1016000040F2F0108B498D4B0B508D48854204D928
:1016100040F2F41087498A4A0A508A48874204D91E
:1016200040F2F8108349874A0A500498032872D080
:10163000049080007F49401840F2BC2142580A9231
:1016400040F28C240259099240F25C25435940F241
:101650002C27C65940F2FC128258411803910119F7
:10166000029141190591C1190791114640F2FC12EE
:1016700080180690019F08371820E7B10C4608999A
:10168000CD19D921695C81400A9A8A180A92A92148
:10169000695C8140099A8A1809927921695C8140C4
:1016A000CB184921695C81408E19697E81400919F6
:1016B00008387F1CE1E707980660069801600598E6
:1016C0000360099F029D2F600A9A039C226064298F
:1016D000594801D3814201D906990860642E01D38B
:1016E000864202D96420079908605448834202D98F
:1016F00052480599086052488742049801D95049D8
:10170000296050498A4201D94E4921600899091D32
:101710000891401C8AE740F20510444F385C40F2C3
:10172000F421444A505040F2F82010180199891DC4
:1017300040F20C1221B17B189B5C08C0891CF9E7B0
:1017400040F21810385C40F21C313A4A505040F2D6
:101750004030101840F21E11791803238BB10C7819
:1017600004600A7B02630CB1642C01D30124046081
:101770000AB1642A01D301220263491C001D5B1EC9
:10178000ECE740F227103A5C40F26431294C625099
:1017900040F23310385C40F29433E0500AB1642ACE
:1017A00002D30122234B5A5008B1642804D340F2DB
:1017B000943001211F4A1150244E0023019AFAB19E
:1017C0002148801801693D46BF1840F240143C5D35
:1017D0002406611840F241143C5D2404611840F273
:1017E00042143C5D2402611840F243143C5D091927
:1017F000B1421F4600D80F460761121D2F46DEE793
:1018000040F2C0300B490818019D093540F25B11C8
:10181000002245B17B195C5C2F2C134600D823466F
:1018200008C06D1CF5E70BB0F0BDC0467C09002078
:10183000000000209C020020B01E0400803801003F
:1018400080B14F01005621837802002000A3E111EE
:1018500070B5154C8021154E2046B047144D2870A8
:1018600040212046B04768700920C406204641F256
:101870000001B047A870204640F20011B047E87060
:101880000C4848F20001B047297809010143687803
:10189000C0000843A97889000143E87842000A4360
:1018A0001F20904370BDC046001400489B1C0008D8
:1018B000B20100200004004870B52220022100F08F
:1018C0004BFC0A20FFF73AF9F04E30798119732268
:1018D0008C5CFFF78BF984420AD17420305A0004E3
:1018E00000BAFEF741FFFEF721FE04460D4603E075
:1018F0000120707100242546F06E0D4902F049FF69
:1019000008B90D4A00E00B4A08B90D4B00E00B4B3B
:1019100020462946FEF7E6FCFEF7A6FC3067306D50
:101920003F21090602F01FFF08B90020306770BD93
:1019300000005C42CFF753E34E621058A59BB43FC2
:1019400039B4B83F70B52820032100F005FC0A2007
:10195000FFF7F4F8CD4D2879411973240E5DFFF798
:1019600045F986420BD17420285C00042946743165
:101970004A781202101889784018A86501E0012001
:1019800068710220014600F0E7FB0A20FFF7D6F855
:10199000287941190C5DFFF729F9844208D1742098
:1019A000285C00022946743149784018E86501E056
:1019B00001206871A86DFEF7D7FE0446286AFEF77D
:1019C000D3FE0146204602F0BBFF3121090602F09A
:1019D000B7FFB04C214602F0B3FF2146FEF7D0FD21
:1019E0002866686670BDC046B0B52420032100F0AB
:1019F000B3FB0A20FFF7A2F8A44D287941197322FE
:101A00008C5CFFF7F3F884420BD17420285C00044F
:101A1000294674314A781202101889784018E86310
:101A200002E001206871E86B010218D4FEF79CFE09
:101A30000446A868FEF798FE0146204602F080FFA3
:101A40000D21890602F07CFF924C2146FEF798FD9D
:101A5000214602F075FF2146FEF792FD00E00020CE
:101A60002864B0BDB0B52320022100F075FB0A2028
:101A7000FFF764F8854D2879411973228C5CFFF7D4
:101A8000B5F884420BD17420285A000400BAFEF73E
:101A90006BFE4121090602F053FF014602E00120DE
:101AA000687100210548FEF76BFD0446784902F095
:101AB00065FE00B10024AC66B0BDC046647A5A4AE7
:101AC000B0B52C20042100F047FB0A20FFF736F8C0
:101AD0006E4D2879411973228C5CFFF787F8844298
:101AE00003D1686F00BAE86402E001206871E86C15
:101AF0000121CA070021904200D9C9434840FEF79E
:101B000033FE04466869FEF72FFE214602F018FFF7
:101B10000321090702F014FF5E4C214602F010FF7A
:101B20002146FEF72DFD2865B0BDC04670B52720C3
:101B3000032100F011FB0A20FFF700F8534E307923
:101B4000811973228C5CFFF751F884420AD174200A
:101B5000305C0004314674314A78120210188978DA
:101B6000441801E001207071306DFEF7DFFC0A4A75
:101B70000A4B02F0EDFD05460120C1058C4201D95A
:101B80000006041B2046FEF7EFFD0549FEF7F8FCB2
:101B900005B10020F06670BD333333333333D33FA8
:101BA000FEFFFF4AB0B52E20042100F0D5FA0A202E
:101BB000FEF7C4FF354D2879411973228C5CFFF77D
:101BC00015F8844203D1686F00BAE86402E001208E
:101BD0006871E86C0121CA070021904200D9C9430D
:101BE0004840FEF7C1FD04466869FEF7BDFD214689
:101BF00002F0A6FE0321090702F0A2FE254C2146B1
:101C000002F09EFE2146FEF7BBFC6865B0BDC046F3
:101C1000B0B52620032100F09FFA0A20FEF78EFFC0
:101C20001A4D2879411973228C5CFEF7DFFF84423C
:101C30000BD17420285C0004294674314A781202C2
:101C4000101889784018686402E001206871686C97
:101C5000010218D4FEF788FD04462869FEF784FDCA
:101C60000146204602F06CFE6921C90502F068FEBB
:101C70000749FEF785FC074C214602F061FE21462C
:101C8000FEF77EFC00E00020A864B0BD3401002017
:101C90000000C84200007A44704780B500F0B9FFE8
:101CA000411E884180BD000070B52D4C02250D4EAF
:101CB00020462946B04700F03BF801212046B047B6
:101CC0002846FEF747FF2046294600F09EFF28469B
:101CD000FEF740FF20462946324670BC08BC9E46AF
:101CE0001047C046072C0008B0B51D4C0225204601
:101CF000294600F088FF00F01BF80121204600F083
:101D000084FF2846FEF726FF2046294600F07DFF87
:101D10002846FEF71FFF20462946B0BC04BC964665
:101D200000F071BF0E48002101230A4600F076BF83
:101D300070B50B4C00250126204631462A46334615
:101D400000F06CFF032220462946334600F085FF51
:101D5000044848F2000170BC04BC964600F053BF32
:101D60000014004800080048F8B504460027CE4D8E
:101D7000084EA7420CD0EB48C15D284602F050F94E
:101D80002846314602F079F90028F9D07F1CF0E7A7
:101D9000F8BDC046060700000348016811B101689C
:101DA000491E01607047C0460C0D002030B4334816
:101DB000026801210A43026002689207FCD542686A
:101DC0002F4B1340436042682E4B13404360026820
:101DD0002D4B13400360C26A0F239A43C262026B09
:101DE00040F203139A4302630A04036B93430363B1
:101DF000CA07036B93430363426B8A434263002227
:101E0000826002680A430260204B022204685D1E61
:101E10009D4202D214402B46F8D003689B0700D4A1
:101E2000FEE71B4B1C680725AC431C601C68144371
:101E30001C60436843604368436043684360436891
:101E4000144C1C4044604368134C1C4344600B0614
:101E500004681C43046003689B01FCD543680324A9
:101E6000A343436043681343436042681207FCD5B1
:101E7000C806002130BC01F045BEC046001002403B
:101E80000C00FF08FFFFC277FFFFF2FEFF04000017
:101E900000200240FFFFC2F70000040810B50A4C02
:101EA0000121204602F062F868B10121204602F0CB
:101EB00059F80021204601F0BBFF0448006810BC1F
:101EC00002BC8E46004710BD0020004024020020C6
:101ED000F8B51C4D01242846214602F047F8012898
:101EE00003D10121284602F03DF836492431002271
:101EF000154B164D032A10D09E5C5EB10E46103E67
:101F000037680868874201D2781C02E0AC54002090
:101F100098543060091D521CECE70D490878294B94
:101F200058B19A68D868824202D2501C986004E086
:101F300008480470002098600870596809B1481E6C
:101F40005860F8BD004001405202002056020020B7
:101F50003F0200204002002010B5074C012120461E
:101F600002F004F8012806D10121204610BC04BC6F
:101F7000964601F0F7BF10BD00440140B0B5104DCA
:101F800001242846214601F0F1FF012803D1012157
:101F9000284601F0E7FF0B480178022901D8491CC7
:101FA00002E009490C70002101700169782902D111
:101FB00006490C7000214470491C0161B0BDC04647
:101FC00000480140000100203802002045020020A6
:101FD000B0B51D4C354D2046294602F07DF830B194
:101FE0001A48006880472046294602F061F8184DDB
:101FF0002046294602F041F8012806D1204629460C
:1020000002F033F8114800688047124D20462946F7
:1020100002F062F830B11048006880472046294637
:1020200002F046F80D4D2046294602F055F848B119
:1020300009480068804720462946B0BC04BC964643
:1020400002F036B8B0BDC046003801401C02002086
:10205000030700000700070720020020060006070C
:10206000B0B5114C114D2046294602F035F8D0B1DB
:102070002046294602F01CF80D4800780D4D2978BD
:1020800081420BD2204601F0C7FF29780B4A5054F9
:102090000B4801220270481C2870B0BD0020287037
:1020A000054801210170B0BD00440040050005074E
:1020B000380100203601002035010020A801002051
:1020C00034010020B0B54048002101710424C470DF
:1020D0003C4D5A20A870EA206870A5202870204640
:1020E000FEF79CFDE8702046B0BC02BC8E46FFF7B0
:1020F0003BBEC046B0B53448002101710424C47011
:10210000304DDC20A870EA206870A5202870204699
:10211000FEF784FDE8702046B0BC02BC8E46FFF797
:1021200023BEC046100D0020B0B527480021017124
:102130000424C470234DE520A870EA206870A5200F
:1021400028702046FEF76AFDE8702046B0BC02BC4D
:102150008E46FFF709BEC04610B51A4A5070A5203A
:102160001070194C0220E070481C2071FEF7D6FC5C
:10217000E07810BC02BC8E46FFF7F6BDBCB5114B33
:10218000A5241C70802404435C700092981C6A464D
:10219000521E0C4624B1155D0570401C641EF9E703
:1021A000094800220271C91CC170CCB2E018451E5A
:1021B0002046FEF733FD28702046BCBC02BC8E468C
:1021C000FFF7D2BD100D002034010020B0B5002073
:1021D000064CA047064D28600120A04768600220F9
:1021E000A047A8600320A047E860B0BD713B00088D
:1021F000B801002010B5144608463F490A220A706B
:102200000722214602F04CF9012804D1044802F0CB
:10221000C5F9012801D0032010BD002010BDC04623
:10222000204E0000F8B506460F4CA088000A16D1D3
:10223000A0880527032810D30D460092A1882648C0
:1022400001F08AFC48B9244908783070481C28609D
:10225000A088801E0099088000273846F8BD03A09A
:102260000C499C22FFF7C6FF2C02002075735263B5
:1022700076427566666572506F73203C204D425FF2
:102280005345525F5044555F53495A455F4D41583D
:1022900000000000C94D0008B0B5174D6B780BB1B8
:1022A000052516E00124EC804B1EAB601870E88811
:1022B0008018E880E988184601F04EFCE9884A1C3D
:1022C000EA80054A5054AC7000252846214601F0AA
:1022D00049FF2846B0BDC0461A0D002010B50120A8
:1022E0000024214601F03EFF03484470204610BC04
:1022F00002BC8E4602F0C2B82C02002080B500203D
:10230000014601F02FFF80BC01BC864601F05EBF94
:1023100010B5064C2078012805D105488068804713
:102320000020207010BD062010BDC0461C000020FB
:1023300004020020F8B50C460988032505292FD191
:102340000279C17809028E18711E89B2314B994207
:1023500026D8811C009187784178002525800123AB
:10236000037023885B1C23805307B2B2D60803B1E5
:10237000761C009B46702088401C20800802C019F3
:10238000401C81B218462B4600F0E8FA20B1F8BC98
:1023900002BC8E4601F0C0BBF0B221880818208034
:1023A0002846F8BDF8B50C460988032505292ED125
:1023B0000279C17809028E18711E89B2154B9942B3
:1023C00025D8811C0091877841780025258002233B
:1023D000037023885B1C23805307B2B2D60803B175
:1023E000761C009B46702088401C20800802C01983
:1023F000401C81B2184600F001FB20B1F8BC02BCC1
:102400008E4601F089BBF0B221880818208028464A
:10241000F8BDC046CE070000F8B50C460988032574
:10242000052923D10279511E7C291FD8831C81786C
:10243000477800252580032606702688761C26808E
:10244000560046702088401C208038024018401CEE
:1024500081B218462B4600F0F7FA20B1F8BC02BC56
:102460008E4601F059BB2088801920802846F8BD8F
:10247000F8B50C4609880325052928D10179C278C9
:10248000120251184A1E92B27B2A20D8821C009256
:102490008778437800252580042202702288521C08
:1024A00022808AB2560046702088401C2080180284
:1024B000C019401C81B2009800F060FB20B1F8BC4C
:1024C00002BC8E4601F028BB208880192080284657
:1024D000F8BDF8B5054608880A2841D30C46287986
:1024E000E97809020F18781E80B203267C2838D8B4
:1024F000287AE97909020818411E89B2782930D86A
:10250000697A82B2500081422BD1A8796979090297
:102510000818411CA87800906E7828460A3089B2C5
:10252000012300F091FAB0B9BAB230020099401814
:10253000411CA81C0026268017232B7023885B1CB7
:10254000238057006F7023885B1C238089B2334639
:1025500000F07AFA38B1F8BC02BC8E4601F0DCBA61
:1025600000263046F8BD2088C0192080F9E7000019
:10257000B0B50C4605490D88401C891C2A46FDF75C
:102580002FFE681C20800020B0BDC046D401002072
:102590001CB50988032405291AD10179C1B98278AB
:1025A0004378C178FF2900D091B918028018421CE5
:1025B00001A800244470FF394B424B41037091B293
:1025C0000122134600F0CAF910B101F0A5FA044641
:1025D00020461CBD80B50988052910D18178427834
:1025E00012025118491C89B2C01C0122134600F086
:1025F0002BFA30B180BC02BC8E4601F08DBA0320AC
:1026000080BD002080BD70B50C460A880321062AD3
:1026100024D30679C27812029519AAB2D308760794
:1026200000D05B1C6D1EADB22D097A2D16D84579F0
:10263000DBB29D4212D1817843781B025918491CA4
:1026400089B2801D012300F089F920B170BC02BC61
:102650008E4601F061BA052020800021084670BD39
:10266000B0B50C460A880321062A20D302794379A3
:1026700055062D0EAB421AD1C3781B029A18531E71
:102680009BB2772B13D8817843781B025918491CC9
:1026900089B2801D92B2012300F0D6F920B1B0BCFE
:1026A00002BC8E4601F038BA052020800021084681
:1026B000B0BD0000F8B50546022091B3CC081E2C31
:1026C0002FD8069C524E3170012D15D04DBB254D93
:1026D0002548264FB760F0603561214870611F487A
:1026E000B0611D48F0611B483062084611461A4629
:1026F000234600F091F813E0134D1448144FB760CF
:10270000F06035610F4870610D48B0610B48F061B1
:1027100009483062084611461A462346FFF76AFD0B
:1027200000B1F8BD01F0A4FE20B1384801210170CC
:102730000020F8BD0320F8BD3943000871430008AC
:102740002D4200082522000899220008FD220008D9
:10275000DD22000885460008D1460008F54500083E
:1027600055280008C9280008492900082D29000813
:102770007CB52648007808B1062445E001A801F0A0
:102780006BFE002401283FD101A80078022812D056
:10279000012839D11E4D6B69681C294624312A1D38
:1027A000984788BB68782978884200D060BB0220AF
:1027B00001F064FE28E0164D6A6A1178A9700023C2
:1027C0000120144C802B0AD0E65C46B18E4201D029
:1027D0000833F7E7E0184368291D104698476978E1
:1027E000002489B158B10121A980A97880220A4327
:1027F000696A0A70A9884A1CAA806A6A5054AA8821
:10280000696A28782B69984720467CBD1C00002007
:10281000040200202000002010B5144608460822BB
:10282000214601F03DFE01280ED144F600308442DD
:1028300001D9232003E060000549B1FBF0F080B22C
:1028400001F0ACFE012801D0032010BD002010BD16
:10285000A07F1700F8B506460F4C6088000A16D115
:1028600060880527042810D30D46009261882E4801
:1028700001F090FB48B92C4908783070481C28605A
:102880006088C01E0099088000273846F8BD03A064
:102890000C499C22FFF7AEFCF801002075735263CF
:1028A00076427566666572506F73203C204D425FBC
:1028B0005345525F5044555F53495A455F4D415807
:1028C000000000006B4D0008B0B51E4D2B78012BA9
:1028D00026D10124AC804B1EAB601870A8888018EC
:1028E000A880A988184601F055FBA9884A1CAA802F
:1028F0000D4A5054A9884B1CAB80000A5054A8685C
:10290000007801F041FEA888401EA880A868401CFD
:10291000A8606C7000252846214601F023FC00E0E9
:1029200005252846B0BDC0461A0D002080B50548D3
:1029300000210170012001F015FC80BC01BC86461D
:1029400001F05CBCF801002080B50020014601F0D8
:1029500009FC80BC01BC864601F038BCFEB51446BB
:102960000246491E88B20019042824D8601E082592
:10297000019590FBF5F0451C0020F3B1012B1BD114
:1029800000901D4B280435D06D1E0292107822460F
:10299000019F541E12040BD03A0609D001220240B6
:1029A0008EB29A55491C7F1EC0B240082246F0E7FD
:1029B000029A521CE6E70120FEBD0090082001901B
:1029C0000D4F280416D002926D1E00262246019853
:1029D000541E12040AD0020608D08AB2BA5CB24071
:1029E0001343761C491C401E2246F1E7029A1370DD
:1029F000521CE6E70098FEBD1A0E0020F0B5491EF5
:102A00008BB2DC0801217D2C1BD39B1840F2EC34E7
:102A1000A34216D8511E082391FBF3F14C1C002150
:102A200025040ED0641E16461D46721E360404D0C0
:102A30006F1E2D0616463D46F7D100250570401C39
:102A4000EEE70846F0BD0000FEB50546481E87B219
:102A5000012002904248874219D91446BE18414AC3
:102A6000964214D841F27072BE1A3F4A5660012B4A
:102A70000FD043BB401C87424CD1022C4AD170007E
:102A80003D490968394A11523A48016052E00298BA
:102A9000FEBD019654700520C04340F2D0734343FD
:102AA0003248C0187B00C3182746164638040CD09D
:102AB0002878000218806A78801832461880AD1C89
:102AC0009B1C7F1EF2E70020FEBD41F2EB70081A4E
:102AD00080B2BB2802981CD80198400023490918ED
:102AE0001078029047012248C5192846083022066E
:102AF000D20DFDF775FB01201D49C8510198686092
:102B00000298411CCAB200200F2A024600D80A4689
:102B10003270FEBD41F2EB70081A793080B2F728AE
:102B20000AD8700011490818B100124A5118620001
:102B3000FDF756FB002000E001200521CA4340F2CA
:102B4000D0715143094A5218790051182204E0D03B
:102B50004A782A700A786A70AD1C891C641EF5E7F1
:102B60006F170000581B0000C80100201E0E002037
:102B70000C0B00209C0200207002002010B50346C0
:102B8000481E81B20120084CA1420BD38918074C82
:102B9000A14207D80020110404D0587018709B1C63
:102BA000521EF8E710BDC046B80B0000BC0B000079
:102BB000FCB50191016A0090446A00252E46202D43
:102BC0000CD01746F740FF0705D0019FAF400F23F9
:102BD000AB40994339432D1D761CF0E708250026AC
:102BE000202E0CD01346EB40DB0705D0019BB340F1
:102BF0000F27B740BC431C43361D6D1CF0E70098FF
:102C000001624462FCBD8162704781617047C162AC
:102C1000704700690840411E88417047FEB5029325
:102C2000019202680090C56800263746202E10D019
:102C3000029BFB40DB0709D0019BB3400324B44057
:102C4000A5431D430B46B340A2431A43B61C7F1C49
:102C5000ECE700980260C560FEBDF8B5012902D11D
:102C60004168194301E041689943416000908168DF
:102C7000002403202646202C0CD01F46F740FF07D7
:102C800005D01746A7400546A540A9433943A41CD3
:102C9000761CF0E700988160F8BD000000B595B0A3
:102CA000EE4F0023BB827B717B70ED4803210F91B7
:102CB00001703020C64330462E30212120B13A1811
:102CC00053545377401CF9E73B721393FB71FFF7A2
:102CD0006DF8FFF77BFAFEF72FF9FEF797F9FEF78D
:102CE0000DF9FEF7DDF8FEF729F9FEF7A3FAFEF776
:102CF000AFF9FEF72BF8FEF715FC42F28050FEF715
:102D000033FAFEF725F80920C0060B900124402075
:102D10001190802010901294D1480078844226D8D7
:102D2000032C13D0022C07D0012C1ED10B9D28465A
:102D30001199FFF76AFF04E00B9D28461199FFF7F0
:102D400062FF28461099FFF760FF08E00B9D2846B8
:102D50001199FFF75AFF28461099FFF754FFC14811
:102D60001299FFF752FFFEF7A7FA641CD4E7FEF7AB
:102D70006FFD0146139C0094E12043022046224649
:102D8000FFF798FCFFF7C4FA40F2F420B64A105857
:102D9000502102917854B549F981116040F2B41183
:102DA00051583A46503201925170C1B22046FEF756
:102DB0009FFB01210B980391FFF725FF2A2414960E
:102DC0002D2C1CD000203855139D7819A64949197F
:102DD00040F2F8268A595423C25489198B6C56261E
:102DE0008355149E896F5723C154D1B22046293888
:102DF000C0B2FEF77DFB2D1D1395641CE0E740F289
:102E00001C30994A10583C21089178540720C0037F
:102E100040F2B41150500024FC7291480F99017097
:102E200040F29430105839463C31C87040F264305A
:102E300010588870388A78828D4940F2341008180A
:102E4000079040F2F8101018069040F2BC301018AD
:102E5000059040F2B8101018049009948348B863A4
:102E6000FDF752FE002800D00BE108983A5C1046AE
:102E7000039B18403873F97A884203D10020B87157
:102E8000397A23E070B90123BB720021797252B202
:102E9000002A0BD53972FB713F22BA5C40F2E8334D
:102EA0005A4310E0BC727B72510604D43B7200227C
:102EB000FA71194607E03C72FB713E217A5C40F2E0
:102EC000E8314A432146F8726A48026041B300245F
:102ED0003C72FC71787A40B120216248FFF795FE80
:102EE0007C720898395C01200AE0B87A68B1202128
:102EF0005C48FFF788FEBC720898395C30462F307A
:102F00000843594940F21C328850564C204644F23E
:102F10000001FFF77AFE204644F20001FFF773FE3E
:102F2000002516271395192F00D1A7E04B4BDC196C
:102F30005E195420315C012208461292104020761E
:102F4000227D824205D1D85D18B300204349C8557F
:102F50001FE0002248B92273129B237449B2002952
:102F60000AD52371227257210CE02274129B23731D
:102F7000490604D440494A512271237208E0237162
:102F800022725621715C40F2E83251433A4A515163
:102F90002075207A002859D01195543600252572C5
:102FA0002571207B58B17F201399084002281AD040
:102FB000012816D0D8B90B9848F2000115E0207C02
:102FC000C0B325747F2013990840022817D0012828
:102FD00013D0119DC0B90B9848F20001FFF713FE02
:102FE00012E0082100E010211E48FFF70EFE2573B5
:102FF000307812990843119D09E0082100E0102162
:103000001848FFF700FE119D307812998843394621
:103010001639154C6219C0B240F2F823D050CAB22A
:103020000F9BB2FBF3F25A43891A3639CF220A407A
:10303000910060500B4C204644F20001FFF7E5FD83
:10304000204644F20001FFF7DEFD119D7F1C2D1D7F
:103050001398401C1390149E65E7C0463802002068
:1030600000000020000400489C020020030800002B
:10307000EC0700200C010020240100200020E94F73
:103080007880FFF775FBFDF7ABFD18B1FEF728FA66
:10309000FDF750FD787B40F24314F8B100207873BF
:1030A0003046253098B1E0490918E04A1218526BB1
:1030B0000A55130A40F242154B55130C40F24115C4
:1030C0004B55120E40F24013CA54001DEAE740F27D
:1030D00005102F300C220799FDF782FC3878002864
:1030E00000D1F7E100243C70032C04D0E0B200F0E2
:1030F000F3FD641CF8E7CE490E6A486A0E90886AB0
:1031000011900B6C4D6C886C0D900A6E4C6E886E35
:103110001290C648466083601392C2600E9A0261A4
:1031200045618461119AC2610D9A02623D4644353F
:1031300034CD0E958D6BAA1811928D6D2A198D6F55
:103140000E996C18129941621199283016C00D968B
:103150009E420C93194600D80D99139EB1423346F6
:10316000B44C00D80B4601210022A3420E91149DBD
:1031700000D311460D980C9B984200D30D9B06B1CD
:103180003346AD48834200D80E920E9808400E9008
:103190003223059813900699A84A2E46A54D362B42
:1031A00000D116E1322B03D01446A448044000E0BD
:1031B0000024322B27D10E98002844D00D98A84225
:1031C0000DD23E461746012298481C462B4640F237
:1031D000983542511D4623463A463746149E0C9870
:1031E000A84200D3EEE03E461746012218462B4681
:1031F00040F2A0358D4C625140F29C358B4C6251AF
:103200001D46034630E012928D48C518AA5D119400
:1032100072B3A20085481218526B0E68B24232D9BE
:10322000149882005618109AB75801200A90074344
:1032300002208743B75013980078800731D579482A
:103240000A9AC2542DE03E461746002277481C4693
:103250002B4640F2A035425140F29C35425140F29B
:10326000983542511D4623463A463746149EA9E0FA
:10327000B00040183446109E875901229743875169
:103280002646119C0EE01498800046181098375876
:103290000F9887438036086B824201D8022007438B
:1032A0003760149E75192879A0B1B0004618803691
:1032B000A0005E4A8018406B0A6B904211D2022037
:1032C000074337601398007840070DD50120554A11
:1032D000D05409E002208743B0004018109A87506C
:1032E00003E0022087433760149E287AA0B1B00023
:1032F00046188036A0004D4A8018806B0A6E9042B6
:1033000011D904200743376013980078C0070DD007
:103310000120444AD05409E004208743B0004018FB
:10332000109A875003E0042087433760149E287B5F
:10333000A8B190200858B20056188036A2003B4C25
:103340001219D26B824211D90820074337601398B3
:10335000007800070DD50120324AD05409E008203A
:103360008743B0004018109A875004E00820874334
:103370003760149E119C287CB8B1C0200858B20058
:1033800055188035A200294C1219D26C824213D9EB
:10339000102007432F6013980078C006214F254D59
:1033A000129A0FD50120F8540CE010208743B0008A
:1033B0004018109A875002E0102087432F60194F61
:1033C0001C4D129A1398001D1390091D08325B1CA6
:1033D000E5E600203946032810D23322362A0AD0E7
:1033E0008B5C521C012BF9D13322362A03D00123E6
:1033F0008B54521CF9E7C91CC01CECE73324002590
:10340000362C4DD0385D002847D02646333E022E5C
:1034100018D0012E04D0CEB90B9848F2000113E069
:10342000082110E038020020EC0700209C02002058
:103430004C07002030750000BFD40100F8FF0000E9
:10344000000000201021FA48FFF7DDFB13957919E1
:103450005422885C0123984388543A19149B9D1880
:103460002C270021E9552833D75C07B1D154F14B03
:10347000139FDA19C0B240F2F82550513D46EE4F85
:103480003955F1B20F9AB1FBF2F15143711A363945
:10349000CF220A4091005850149E2D1D641CAFE7A6
:1034A000E34C204644F20001FFF7AFFB204644F214
:1034B0000001FFF7A8FB388A0021049A032908D0ED
:1034C00001238B4010CA0CB1184300E09843491CFB
:1034D000F4E7388278794101D84B5A58002A00D154
:1034E0008EE259184D6828467A38BB2800D981E207
:1034F0008C68810001A251188F46C04600F076B951
:1035000000F074B900F072B900F070B900F06EB953
:1035100000F06CB900F06AB900F068B900F066B963
:1035200000F064B900F062B900F060B900F05EB973
:1035300000F05CB900F05EBA00F05CBA00F05ABA74
:1035400000F054B900F052B900F050B900F04EB993
:1035500000F04CB900F04AB900F048B900F046B9A3
:1035600000F044B900F046BA00F044BA00F042BAA4
:1035700000F03CB900F03AB900F038B900F036B9C3
:1035800000F034B900F032B900F030B900F02EB9D3
:1035900000F02CB900F02EBA00F02CBA00F02ABAD4
:1035A00000F024B900F022B900F020B900F01EB9F3
:1035B00000F01CB900F01AB900F018B900F016B903
:1035C00000F014B900F016BA00F014BA00F012BA04
:1035D00000F00CB900F00AB900F008B900F006B923
:1035E00000F004B900F002B900F000B900F0FEB834
:1035F00000F0FCB800F0FEB900F0FCB900F0FAB938
:1036000000F0BFB900F0CEB900F0E0B900F001B9A8
:1036100000F0FFB800F0FDB800F0FBB800F0F9B81A
:1036200000F0F7B800F0F5B800F0F3B800F0F1B82A
:1036300000F0EFB800F0DEB900F0DCB900F064B9DA
:1036400000F062B900F060B900F0D4B900F0D2B96E
:1036500000F0D0B900F0E4B800F0E2B800F0E0B853
:1036600000F0DEB800F0DCB800F0DAB800F0D8B84E
:1036700000F0D6B800F0D4B800F0D2B800F0BAB973
:1036800000F0B8B900F0DCB800F0DAB800F0D8B853
:1036900000F0D6B800F0D4B800F0D2B800F0D0B83E
:1036A00000F0CEB800F0CCB800F0CAB800F0A2B973
:1036B00000F0A0B900F09EB900F09CB900F09AB9F2
:1036C00000F098B900F096B900F094B900F092B902
:1036D00000F090B900F0C4B800F0C2B800F0C0B873
:1036E00000F0BEB800F0BCB800F0BAB800F0B8B84E
:1036F00000F0B6B800F0B4B800F07CB900F07AB9C8
:1037000000F078B900F076B900F074B900F072B941
:1037100000F070B900F06EB900F06CB900F06AB951
:1037200000F068B900F066B900F064B900F062B961
:1037300000F060B900F05EB900F05CB900F05AB971
:1037400000F058B900F056B900F054B900F052B981
:1037500000F050B900F04EB900F04CB900F04AB991
:1037600000F048B900F046B900F044B900F042B9A1
:1037700000F040B900F03EB900F03CB900F03AB9B1
:1037800000F038B900F036B900F034B900F032B9C1
:1037900000F030B900F02EB900F02CB900F02AB9D1
:1037A00000F028B900F026B900F024B900F022B9E1
:1037B00000F020B900F01EB900F01CB900F01AB9F1
:1037C00000F018B900F057B800F055B800F053B841
:1037D00000F051B800F04FB800F04DB800F04BB811
:1037E00000F049B800F047B800F013B9A800A249AA
:1037F0000C50A3494018210EA24A11541118220C52
:103800004A70220A8A70CC7080B20422FDF7E8F870
:10381000EFE02E46BE3E092E61D108983C5467E089
:10382000D92D03D0A800C019994944543E200EE078
:10383000000400489C020020380200200C0B0020ED
:10384000E52D03D0A800C019904944543F203C54B2
:10385000A8004E358B494C55E1B2874A115006E01D
:10386000A800E1B2844A1150683586484455A8B290
:10387000FDF7C6F8BDE0002C00D1BBE0A8007F49F1
:10388000401800227F4B1A547D4949198900C919F3
:1038900040F230340A5119184A708A70CA7080B2E6
:1038A0000422FDF79DF83046253040F2431380B1E5
:1038B000744909180022CA5440F242140A5540F2D1
:1038C00041140A5540F240140A553918CA64001DC3
:1038D000EDE740F205102F300C22079996E7BD3D29
:1038E000A800381802994454E1B2E8B2FDF700FE8E
:1038F000700040F20611401862490C5480B2E1B2E7
:10390000FDF77EF8149E74E0CA3D0F986843411C91
:103910008A00019EB4547A1901239375821C0E9279
:103920009700F455C01C1290800011903454C8B216
:10393000E1B21391574A9047F15D0E98C0B24D4FD6
:10394000544A90471198315C1298C0B2514A90473E
:103950000620684340F206114018851C49494C5521
:103960000C54061D8C5580B213994B4CA04745480A
:10397000415DA8B2A0474348815DB0B2149EA04704
:1039800037E00120B87040F206103E490818542173
:10399000602941D00278412313437B540370091DF1
:1039A000801CF5E70120F87040F206103549081830
:1039B0005421602943D002787E2313407F22D243D2
:1039C0009A187A540270091D801CF2E740F2051023
:1039D0002C490C54029D7C55274840F2F421445058
:1039E000E1B240F20510FDF70BF8795D0020FDF71C
:1039F0007FFD254B7879410100225A500121397110
:103A0000401CC1B20F2900D90020099C7871FFF732
:103A100025FA002CEED046E740F20610194C21188A
:103A200040F20510401C0622FCF7DAFF40F21812A3
:103A3000A05C4121014308983954A15414E040F29C
:103A40000610104C211840F20510401C0622FCF70D
:103A5000C7FF40F21812A05C7E2101407F20C043C6
:103A6000081808997854A054A11840F20510133092
:103A70000222CBE6380200209C02002084FCFFFFDB
:103A800019FEFFFFEC0700200C0B0020E7FCFFFFF6
:103A900016FDFFFFF1140008010A000870B540B2DE
:103AA000002817D4032302469A43144BD4588507A1
:103AB000ED0EFF26AE40B4438901C9B2A9402143AF
:103AC000D1501F21014001228A40400980000C4949
:103AD000425070BD8207D20EFF2494400F23034052
:103AE000083B0320834304481D58A5438901C9B2FC
:103AF00091402943195070BD1CED00E000E400E046
:103B000000E100E0024A0A400243024802607047B6
:103B100080FFFF1F08ED00E040B1072803D0012817
:103B200003D1022070470620704704207047000030
:103B30000A2801D2302102E0102803D237210818C8
:103B4000C0B2704702A0034940F2D012FEF752FB08
:103B500030000000C94D000800220B0405D0037896
:103B6000D218D2B2401C491EF7E75042C0B270478B
:103B7000F8B501463E4B18680C2202403D48082A21
:103B8000044618D11A689202120F0F2A01D0941C11
:103B900000E010241D682D0101D5113214461A6869
:103BA000D20301D4344A05E09A6A0F2515406A1CF5
:103BB000B0FBF2F254431D6818681A6805291FD833
:103BC00000902D062D0F2DA77F5D2546FD40920408
:103BD000520F2E4FBE5C2A46F2408E0001A0801983
:103BE0008746C04600F00AB800F011B800F00AB8E5
:103BF00000F00EB800F00EB800F014B8224607E04E
:103C0000002205E000984005400F385CC5402A4678
:103C10001046F8BDD86AC0051AD4D86AC00320D5AA
:103C20001C48F8BDD86A8007F2D0D86A0321084042
:103C300001282246ECD0D86A084048F20002022847
:103C4000E6D0D86A084003280A4800D00020F8BD12
:103C500018680004800FD96A002904D4B2FBF0F27E
:103C6000D6E70B48F8BD401CB5FBF0F2D0E7C046E4
:103C70000410024000127A0000093D00000000001C
:103C8000000000000102030406070809004D0008B7
:103C9000809FD500003FAB011F21014001228A40D7
:103CA00080090C4943581343435070471F2101407A
:103CB00001228A4080090749435893434350704783
:103CC0001F21014001228A408009024943581343C1
:103CD0004350704700100240FEB50446401C4F4F51
:103CE000B871022C0CD0012C16D0002C00D094E01E
:103CF00002900920C50640212846FEF786FF12E003
:103D000002900920C50640212846FEF77EFF80214B
:103D10002846FEF778FF0AE002900920C5064021F8
:103D20002846FEF770FF80212846FEF76EFF3C48CC
:103D30000121FEF76AFFFCF783FEB86C394D294676
:103D400000F0FEFDFCF7CCFC1F2800D20020B97962
:103D50004901354A50505618386C294600F0F0FD9C
:103D6000FCF7BEFC70601E2804D8301D00250560DD
:103D700028460CE0386D2B4900F0E2FDFCF7B0FC62
:103D80000546786D274900F0DBFDFCF7A9FCE10052
:103D900001913061B5606DB1386DFC6E2146FCF764
:103DA000EFFB796D00F024FE1E4900F0C9FDFCF721
:103DB00097FC01E0FC6E0020F060B86E194D2946BA
:103DC00000F0BEFDFCF78CFC7061386E294600F0F7
:103DD000B7FDFCF785FCB0612046294600F0B0FD38
:103DE000FCF77EFCF061029840010F490A580292EC
:103DF000019AD2B292000D4BD2180818071DF8CFC5
:103E00008169C0690190029850639363D46315641B
:103E100056649764D16401981065FEBD340100209A
:103E20000004004800007A444C0700209C02002057
:103E30004162704710B5154C4449884213D014496B
:103E4000884212D0EC49884211D03D49884213D0B3
:103E50003D4988420DD03E4988420CD039498842BC
:103E600013D1F63408E0E41D06E0F93404E0FD3433
:103E700002E0641D00E0A41D2046FFF721FF20465C
:103E800010BC02BC8E46FFF711BF10BD0B03000033
:103E900000100040016801229143016070470168F1
:103EA00001220A430260704710B50A888262244AE0
:103EB000904202D0234B98420BD103687024A34355
:103EC00003604B8804681C4304608B8804681C43AF
:103ED00004608B68C36290420FD1136840F20034D3
:103EE000A3431360CB8814681C431460097B0163EF
:103EF000416901220A43426110BD124A90420BD02F
:103F0000C94A904208D0104A904205D00F4A9042C8
:103F100002D00F4A9042EBD1026840F200339A433C
:103F20000260CA88036813430360074A9042DDD0E9
:103F3000074A9042DAD0054A9042D7D0D8E7C04627
:103F4000002C0140000400400040014000480140B6
:103F500000440140C2688A43C2607047C2680A4395
:103F6000C260704702698A4302617047C2680A40B2
:103F7000531E9A4100690840411E88411040704715
:103F80000349002202730260426081607047C046AC
:103F9000FFFF0000F0B5FF24094A0A4B25460E0436
:103FA00009D006787540565D5F5D25467D40401C12
:103FB000491E3446F3E72002284380B2F0BDC046D4
:103FC000004C0008004B0008B0B50D4604467E4882
:103FD000844204D02048844205D1022000E005201C
:103FE000FFF7C6FD00E000202168090405D4690838
:103FF0004018B0FBF5F080B209E0690840004018B5
:10400000B0FBF5F0034901400007400F4018E060A5
:10401000B0BDC046F0FF0000416A03480840704749
:10402000014A0A4082627047FF01000010B56649EC
:10403000884204D0084988420BD1084C00E0054C66
:104040002046FFF73DFE204610BC02BC8E46FFF71F
:104050002DBE10BD0E0300000044004011040000FE
:10406000016801220A43026070471F220A400121B1
:104070009140026A0A43026270471F220A4089097E
:104080000958D1400120084070471F220A400123EF
:10409000934089090A589A430A5070471F220A40E0
:1040A0000123934089090A581A430A5070470000B7
:1040B000084A914206D1D021425848F200039A435F
:1040C00042507047C902C90E01228A40016A114359
:1040D0000162704709340F341F220A400B049B0D04
:1040E0001B58D3408A0D1258C802C00EC2401A4055
:1040F000012010407047026801239A430260026861
:1041000040F200639A43026002680A43026070470B
:10411000026804239A43026002680A4302607047FF
:10412000026801239A430260426843F200039A4303
:10413000426042680A4342607047026808239A431B
:10414000026002680A4302607047026801239A43D2
:104150000260026841F200039A43026002680A4367
:104160000260704770B50E460921CC06CB4D052183
:10417000012808D12846FFF791FF204640F60001AC
:10418000FEF741FD07E02846FFF77FFF204640F697
:104190000001FEF73AFD06212846012E09D1FFF75E
:1041A0007DFF204640F6000170BC04BC9646FEF739
:1041B0002CBDFFF76AFF204640F6000170BC04BC2E
:1041C0009646FEF720BDC04600380140B0B5164CFB
:1041D00000212046FFF72CFE012520462946FFF747
:1041E000C1FE20462946FFF7B5FE2046B0BC02BC02
:1041F0008E46FFF74FBEC04600200040B0B50A4CC7
:1042000000212046FFF714FE012520462946FFF72E
:10421000A9FE20462946FFF7A1FE2046B0BC02BCFD
:104220008E46FFF73CBEC04600200040BCB53A4D6C
:10423000A87800286AD101A800F028F9687800243D
:1042400078B1022818D001285ED1FFF7D7FF01A866
:1042500000780D2828D000243A2828D1EC70AC80B2
:1042600052E001A800783A284ED1FFF7C7FF00249A
:10427000AC80EC70012018E001A800782978884211
:1042800008D1FFF7A3FF00206870012000F0F6F8C6
:10429000044639E000243A2810D1EC70AC800120AB
:1042A0006870FFF7ABFF2FE0022068702CE001463A
:1042B0004139C9B2062903D3E14303E06C7023E01E
:1042C000014637393038C2B20A2A00D30846E978A5
:1042D00001290AD0C1B9A988FF2911D8A9880001EC
:1042E000E74A50540120E8700EE0A988E44A535C84
:1042F00003435354A888401CA8800024EC7003E0BA
:1043000000246C70FFF762FF2046BCBD03A051493A
:10431000E322FDF76FFFC0462C02002065536E6458
:104320005374617465203D3D2053544154455F549E
:10433000585F49444C45000080B53E484178491ECD
:10434000012902D80021417005E04178012902D0FD
:104350004078022803D1FFF739FF002080BD0348D1
:104360003C4940F2A712FDF745FFC046854D0008C5
:1043700070B5304E7078002856D1B078042840D8F7
:10438000810001A251188F4600F008B800F027B84C
:1043900000F009B800F02BB800F014B8012000219B
:1043A000FFF7E0FE2DE0F08830B3F07801282AD046
:1043B00038BBB06800780009FFF7BAFB00F0E4F8FA
:1043C000012012E00024B470032000F057F80546E5
:1043D00001202146FFF7C6FEB470284670BD3A2082
:1043E00000F0D2F80220B0700020F07009E03078C0
:1043F00000F0CAF8042003E00D2000F0C5F8032007
:10440000B070002070BDB06801780F200840FFF741
:104410008FFB00F0B9F80020F070B068401CB0606D
:10442000F088401EF080ECE703A00A4940F24F12EA
:10443000FDF7E0FE2C020020655263765374617430
:1044400065203D3D2053544154455F52585F4944D7
:104450004C450000C94D00080B490A78012A05D1D6
:104460004A780270002008700120704700207047D1
:1044700005480021017001207047C046024948707C
:10448000012008707047C046D001002010B50446D6
:104490004148FFF7C1FD2070012010BD00380140E8
:1044A000FEB502911B2000252946FFF7F7FA334895
:1044B000FFF7F2FB0920C60601243046214640F2F0
:1044C0000022FEF775FB022101913046224640F2A0
:1044D00000232B4FB8472B4F30462946224640F247
:1044E0000023B8473046214640F20042FEF760FB09
:1044F00030460199224640F20043214FB8473046EA
:104500002946224640F200431E4FB8473046214616
:104510002A4640F600031A4FB84703223046294680
:1045200040F60003174FB847304640F60001FEF74B
:104530006AFB1248FD30FFF7AFFB174E3046FFF71E
:1045400075FD30460299FFF73FFD30462946FFF7DB
:10455000E7FD30462946FFF7F8FD30462946FFF7CC
:10456000CAFD04213046FFF7D3FD08213046FFF78E
:10457000E4FD3046FFF774FD2046FEBD1105000046
:104580001D2C00085B2C000880B501460248FFF78F
:1045900047FD012080BDC046003801407FB505467B
:1045A00040F20870FFF778FB104C2046FFF742FC02
:1045B0006E463046FFF7E4FC0D483080681E0290DE
:1045C0000020019020463146FFF76EFC0125204671
:1045D0002946FFF7C3FC13202946FFF75FFA204660
:1045E000FFF75DFC284604B070BDC04600200040C7
:1045F0000F0E00001CB51A4C607858BB01A8FFF7DD
:1046000045FF2078032823D8810001A251188F4646
:1046100000F01CB800F004B800F00CB800F016B8B8
:10462000002060806088411C61801549019A0A540D
:1046300002200AE06088FF2806D86088411C61805B
:104640000F49019A0A5401E003202070FFF7D6FDBC
:1046500000201CBD03A03D49F022FDF7CBFDC04664
:10466000F801002065536E645374617465203D3D0C
:104670002053544154455F54585F49444C45000011
:104680001A0D0020B0B5294D28780024032808D041
:10469000022802D058B9002000E00120FFF7EEFE0A
:1046A0000446FFF793FD012028702046B0BD28780E
:1046B0000028F6D028780228F3D028780328F0D0F4
:1046C0000248224940F26512FDF794FD084D0008AA
:1046D00070B5164E3078012822D17078012805D0A7
:1046E00080B901200021FFF73DFD0BE0B08858B1F3
:1046F000B0680078FFF748FFB068401CB060B08831
:10470000401EB080002070BD0320FFF7B7FE0446B6
:10471000012000252946FFF725FD7570204670BD54
:1047200003A00A4940F22B12FDF764FDF8010020B6
:10473000655263765374617465203D3D2053544146
:1047400054455F52585F49444C4500006B4D00088A
:1047500010B500F029F8EFF30080800001D40120AB
:1047600010BD002010BD10B500F096F8EFF30080EA
:10477000800001D5012010BD002010BD10B500F053
:104780008BF8EFF300804000800F012800D000205C
:1047900010BD10B500F0AAF8EFF30080800001D43E
:1047A000012010BD002010BD70B501252D050C00A5
:1047B0001C4310D4EC4206D4AC420AD4994200D037
:1047C00070BD904270BDE94217D4EB4215D49942B6
:1047D00070BD894270BDEC4206D5AC42F9D58B4222
:1047E00000D070BD824270BD6D004C00EC4204D21E
:1047F0005C00EC4201D28B4270BD034C30B4FBF73D
:10480000B7FF30BC70BD00BF1900160470B501259C
:10481000ED0704004C4020D4441A01D2001B0919B2
:10482000C60D4B00F2B2FF2A29D01B0E2CD000027D
:104830000C0228432C43D31ADC40051910D2280A55
:1048400002D3401C6D0611D0761EF6058019FF2A92
:1048500000DA70BDC00DC00570BD694000F0CEF833
:1048600001200543C541521C761CE8E764089C40C2
:10487000C90161408900E7D10124A043E4E71B0E90
:10488000440200D0034870BD002AFCD1C00FC0070D
:1048900070BD00BF0000C07F0123DB0502000A439A
:1048A0000DD4DA4203D49A4207D488427047D842E2
:1048B00014D4D94212D48842704780427047DA42F9
:1048C00003D59A42F9D5814270475B004200DA4233
:1048D00004D24A00DA4201D28142704710B5024A3E
:1048E000FBF796FF10BD00BF090013040123DB0591
:1048F00002000A430DD4DA4203D49A4207D4884214
:104900007047D84214D4D94212D4884270478042AA
:104910007047DA4203D59A42F9D5814270475B006D
:104920004200DA4204D24A00DA4201D281427047A0
:1049300010B5024AFBF76CFF10BD00BF090016045A
:1049400070B5420064414B005C41120E39D01B0E21
:1049500038D0FF2A3CD0FF2B3AD0D2187F3A400201
:104960004902400A490A4518ED0106004E43000A73
:10497000090A48430104731A4019190C4318990F86
:1049800004D05B08012149075B1A521CD80904D3E3
:10499000401CF50301D19D0607D0FF2A08D2D5059A
:1049A00006D0E4072043401970BD0125A843F4E771
:1049B000002A01DCE00770BD2402FF202043C0056F
:1049C00070BD1B0EFF2A03D0FF2B01D0E00770BD86
:1049D000FF2636064500B54206D84D00B54203D83D
:1049E000D218FF2A00D0E7E7004870BD0000C07F62
:1049F00070B50125ED0704004C4022D4441A02D2C0
:104A00006C40001B0919C60D4B00F2B2FF2A4BD0B7
:104A10001B0E50D000020C02A8432C43D31ADC40DA
:104A2000051B05D5AD0019D36D08761E521E37D073
:104A3000F605280A01D2801970BD70416D0603D0B9
:104A400070BD6940FFF7E8FE9C40090261404900E3
:104A500001D0401E70BD0124A04370BD6D081DD063
:104A600001202B0C01D12D0410302B0E01D12D0271
:104A700008302B0F01D12D01001DAB0F01D1AD006E
:104A8000801CEB0F01D16D00401C361A121A6D000C
:104A9000680AF5054019012A02DB70BD002070BDCF
:104AA000C036300AC00770BD1B0E440201D1FF2B77
:104AB00000D1024870BD002AF0D070BD0000C07F58
:104AC0008182838485868788898B8C8D8E8F919255
:104AD00093959697999A9C9D9FA0A2A3A5A7A8AAF3
:104AE000ACAEB0B2B3B5B7B9BCBEC0C2C5C7C9CC15
:104AF000CED1D4D7D9DCDFE2E6E9ECF0F3F7FAFE69
:104B000000C1814001C0804101C0804100C181409D
:104B100001C0804100C1814000C1814001C080418D
:104B200001C0804100C1814000C1814001C080417D
:104B300000C1814001C0804101C0804100C181406D
:104B400001C0804100C1814000C1814001C080415D
:104B500000C1814001C0804101C0804100C181404D
:104B600000C1814001C0804101C0804100C181403D
:104B700001C0804100C1814000C1814001C080412D
:104B800001C0804100C1814000C1814001C080411D
:104B900000C1814001C0804101C0804100C181400D
:104BA00000C1814001C0804101C0804100C18140FD
:104BB00001C0804100C1814000C1814001C08041ED
:104BC00000C1814001C0804101C0804100C18140DD
:104BD00001C0804100C1814000C1814001C08041CD
:104BE00001C0804100C1814000C1814001C08041BD
:104BF00000C1814001C0804101C0804100C18140AD
:104C000000C0C101C30302C2C60607C705C5C4046C
:104C1000CC0C0DCD0FCFCE0E0ACACB0BC90908C8DC
:104C2000D81819D91BDBDA1A1EDEDF1FDD1D1CDCCC
:104C300014D4D515D71716D6D21213D311D1D0103C
:104C4000F03031F133F3F23236F6F737F53534F42C
:104C50003CFCFD3DFF3F3EFEFA3A3BFB39F9F8389C
:104C600028E8E929EB2B2AEAEE2E2FEF2DEDEC2C8C
:104C7000E42425E527E7E62622E2E323E12120E0FC
:104C8000A06061A163A3A26266A6A767A56564A4EC
:104C90006CACAD6DAF6F6EAEAA6A6BAB69A9A8685C
:104CA00078B8B979BB7B7ABABE7E7FBF7DBDBC7C4C
:104CB000B47475B577B7B67672B2B373B17170B0BC
:104CC00050909151935352929656579755959454AC
:104CD0009C5C5D9D5F9F9E5E5A9A9B5B995958981C
:104CE000884849894B8B8A4A4E8E8F4F8D4D4C8C0C
:104CF000448485458747468682424383418180407C
:104D000000000000010203042820655263765374FA
:104D1000617465203D3D2053544154455F52585FB6
:104D2000494E49542029207C7C20282065526376F6
:104D30005374617465203D3D2053544154455F5286
:104D4000585F5243562029207C7C202820655263DE
:104D5000765374617465203D3D2053544154455F42
:104D600052585F4552524F522029002E2E2F41702B
:104D7000702F4D6F646275732F7274752F6D627230
:104D800074752E63002820655263765374617465D0
:104D9000203D3D2053544154455F52585F52435685
:104DA0002029207C7C20282065526376537461740E
:104DB00065203D3D2053544154455F52585F574153
:104DC00049545F454F462029002E2E2F4170702FE9
:104DD0004D6F646275732F61736369692F6D6261D2
:104DE000736369692E630000084E0008000000200C
:104DF000A000000010010008A84E0008A00000203C
:104E0000501D00002C0100080301000000010000FB
:104E1000000100000001000000010000000000008F
:104E200000A24A04020000001100000071250008E1
:104E30000400000071240008030000001924000889
:104E4000100000006126000806000000D5250008BB
:104E500017000000D32400080100000035230008DB
:104E600005000000912500080F000000072600083B
:104E700002000000A5230008000000000000000060
:104E80000000000000000000000000000000000022
:104E90000000000000000000000000000000000012
:084EA00000000000000000000A
:04000005080001A945
:00000001FF
